:1000000000308A00C92900000A108A100A118207EC
:1000100028340C34013406340A108A100A1182077D
:10002000413468346F346A3400341C308400000872
:100030000319292801308D008C018C0B1D288D0B94
:100040001C284A308C008C0B232800000000800BF9
:100050001A2800340608C339A300220D8C008C0D29
:10006000FC308C050C083C392304860006148316EA
:100070000610000083120610831606108312003447
:10008000A008031D4528861046288614831686106E
:100090008312A10E2108A2002A20A10E2108A2008D
:1000A0002A200D308C008C0B5328003414309C0017
:1000B0001520C3308316860583128610831686109A
:1000C0008312061083160610831299011908023C48
:1000D000031C722802309C0015200330A2002A2045
:1000E000990A66280D308C008C0B74280230A2000F
:1000F0002A200D308C008C0B7B2899011908023CBA
:10010000031C8E28190804209A00A0011A08A100D7
:10011000402002309C001520990A7E28CD2901300C
:100120001C029E001D08023C031D982840309E07BB
:100130001E0880389F00A0011F08A1004020003445
:100140001B088C000C300C020319B3280A300C0277
:100150000319BB280D300C020319C12808300C020A
:100160000319C628CB28A0010130A100402002308D
:100170009C001520D72801309C0002309D008F2064
:10018000D72801309C009D008F20D728A001103077
:10019000A1004020D7281B081F3C031CD128073092
:1001A0009B050130A0001B08A1004020D728003487
:1001B0001E088400800104309F009F080319EE2868
:1001C000831685158312851DE72804309F0029308A
:1001D0008C008C0BE92800009F03DD288316851511
:1001E0008312851DEE28DD308C008C0BF528000075
:1001F00000001D08840083168515003083128519C0
:10020000013080009F011F08033C031C2329A630F6
:100210008C008C0B092900001E0884000310000CC0
:100220008C008000831685158312851D1C291E08ED
:10023000840008300007800006308C008C0B1E29DB
:1002400000009F0A032900308D0000341B309D0000
:100250001A089E00D8208D080319312901308D001D
:1002600081299B08031D26291A08840000080F3CD9
:1002700003193D2902308D0081291B309D0019088A
:100280009E00D8208D080319482901308D0081294E
:100290009B08031D4E2903308D0081291B309D00D2
:1002A0001A089E00D8208D080319592901308D00A5
:1002B00081299B08031D5F2903308D0081291B3094
:1002C0009D001C309E00D8208D0803196A2901303A
:1002D0008D0081299B08031D702903308D00812921
:1002E0001908840000089D001A08840000081D07F2
:1002F0000F391C0203197F2903308D00812900303A
:100300008D00F5291C088D011B0203188A291B0882
:100310008C0096298C0108309D009B0D8C0D1C08CB
:100320000C0203188C008D0D9D0B8D2900340D08D7
:1003300019089B0064309C0082210C0899000D086C
:100340003030031DAA291A189A159A19B0291A1AB9
:100350002030AC299A111A128D070D089B00A0209D
:1003600019089B000A309C0082210C0899000D0896
:100370003030031DBF299A19C3291A1A20308D075E
:100380000D089B00A0203030990719089B00A02081
:10039000003484011F308305562805309C00152049
:1003A000990119080C20990A9B00A0200430190219
:1003B000031DD12903309A002E309B00A0209A0BF8
:1003C000DC290230990096309C001520990BE32916
:1003D0008E018F0191019201930194019501960183
:1003E0001730990018309A0026298D080319FA2928
:1003F000930AAA2A01301702FD3E03180C2A033E75
:10040000AC2A18088E00910A0C2A18088F00920A4C
:100410000C2A180890000C2A01309C009D008F20A7
:1004200058309B00A0200E08990011309A009721A7
:1004300020309B00A0201108990010309A009721CD
:100440001308990010309A00972114089900103071
:100450009A00972120309B00A02020309B00A020F4
:1004600001309C0002309D008F2059309B00A0205D
:100470000F08990011309A00972120309B00A0208E
:100480001208990010309A00972115089900103031
:100490009A0097211008990010309A009721203077
:1004A0009B00A02020309B00A02083160511831202
:1004B000051501309C0015200E08980018089803B7
:1004C000003A03196D2A15308C008C0B652A000048
:1004D0009808031D6C2A00305E2A831605118312CA
:1004E0000511831606108312061401309C00152096
:1004F0000F08980018089803003A0319892A153044
:100500008C008C0B812A00009808031D882A00307B
:100510007A2A83160610831206100E081E3C8D00E0
:100520000F080D02980018089803003A0319A22A30
:1005300015308C008C0B9A2A00009808031DA12A04
:100540000030932A9018A62A0511A72A05158316AC
:1005500005118312F02963000A108A140A11820718
:06056000012A052A092A08
:02400E00F13F80
:00000001FF
